:100000000C9487050C94CF050C94CF050C94CF0568
:100010000C94CF050C94CF050C94CF050C94CF0510
:100020000C94CF050C94CF050C94D1130C94CF05F0
:100030000C94E9210C94CF050C94CF050C94CF05BA
:100040000C94CF050C94CF050C94CF050C94CF05E0
:100050000C94CF050C9442220C94CF050C94CF0540
:100060000C94CF050C94CF050C94CF050C94CF05C0
:100070000C94CF050C94CF050C94CF050C94CF05B0
:100080000C94CF050C94CF050C94CF050C94CF05A0
:100090000C94CF050C94CF050C94CF050C94CF0590
:1000A0000C94CF050C94CF050C94CF051F1246126B
:1000B0003E1346123E139212B5123E130C131B133D
:1000C0001D181D1855185518D0180419FB1AFB1ABD
:1000D0001B19FB1AAC18AC18B51AFB1ACA1AE81A85
:1000E000041607090B0A1D1B06196405141A0815C6
:1000F0001C171E1F202123222E26242D25273012D7
:10010000182F0C13280F0D340E33313638111037D9
:100110002B2C352A5829787B79397A504F515272D5
:100120006C6368566D668053020103555880576DA5
:100130006E5462595A5B5C5D5E5F6F606174756698
:100140003E3F403C4142774476466B47804365459D
:100150003248494A4B4C3D4D3B4E3A7D7E7C7F7345
:100160004552524F523A206D65646961206B657942
:10017000300A004552524F523A206D656469612041
:100180006B6579310A006D3A2530345820002530EE
:10019000345820004D3A646574656374206167616A
:1001A000696E0A00544D353A206578740A00556E20
:1001B0006B6E6F776E0A00544D353A206465666148
:1001C000756C740A005D206370693D25640A002522
:1001D00030325820004578743A205B00436C6173DC
:1001E000736963203230306370690A00436C617355
:1001F000736963203130306370690A004D3A61647D
:100200006472256420726567333A20253034580AB9
:10021000004D3A6D6F7665206661696C0A004D3A53
:1002200061646472256420726567333A2025303436
:10023000580A004D3A5B423A2530325820583A2548
:10024000642825642920593A2564282564292041F9
:100250003A25645D0A004D3A5B253032582025303E
:10026000325820253032582025303258202530325F
:10027000585D0A0020616464723A25642C2072651E
:1002800067333A253034580A000A5363616E3A0ADC
:10029000004D65646961206B6579730A0068616E61
:1002A000646C65723A20253032582C2049534F3AFD
:1002B0002025730A000A4B6579626F6172643A0AFD
:1002C000007300530052000A4B6579626F617264DB
:1002D0002073746172742E0A000A55534220636FB2
:1002E0006E666967757265642E0A000A0A544D4B82
:1002F0003A61333665666639322F4C5546410A0AF3
:10030000002E0341004400420020006B006500798C
:100310000062006F00610072006400200063006FE3
:10032000006E0076006500720074006500720000C7
:10033000000E0374002E006D002E006B002E0000D6
:10034000000403090409027400040100A032090436
:1003500000000103010100092111010001224000F8
:100360000705810308000A090401000103010200D6
:10037000092111010001224D000705820308000A2E
:1003800009040200010300000009211101000122FB
:1003900036000705830308000A090403000203006E
:1003A0000000092111010001222200070584032019
:1003B00000010705040320000112011001000000E4
:1003C00008EDFEDB0A0101010200010631FF09749C
:1003D000A1010975150026FF009520750881020905
:1003E00076150026FF00952075089102C0050109C9
:1003F00080A10185021601002637001A81002AB764
:1004000000751095018100C0050C0901A10185034B
:10041000160100269C021A01002A9C027510950103
:100420008100C005010902A1010901A10005091906
:1004300001290515002501950575018102950175B4
:100440000381010501093009311581257F95027568
:1004500008810609381581257F95017508810605F3
:100460000C0A38021581257F950175088106C0C0E8
:1004700005010906A101050719E029E71500250175
:10048000950875018102950175088101050819011A
:1004900029059505750191029501750391010507DF
:1004A000190029FF150026FF00950675088100C078
:1004B000636F6E73756D65723A20253034580A008B
:1004C00073797374656D3A20253034580A000A0038
:1004D0002530325820006B6579626F6172643A2072
:1004E000004C45443A20253032580A0025583A2518
:1004F00030386225730A000A202030313233343517
:1005000036370A00290A002575002F002575005D81
:1005100028002564002000256400200025640020B8
:10052000002564007C0025303258006D6F757365BE
:100530006B6579205B62746E7C7820792076206808
:100540005D287265702F61636C293A205B006D6BCA
:100550005F776865656C5F74696D655F746F5F6D0B
:100560006178203D2025640A006D6B5F77686565C2
:100570006C5F6D61785F7370656564203D202564F4
:100580000A006D6B5F74696D655F746F5F6D617894
:10059000203D2025640A006D6B5F6D61785F73708C
:1005A000656564203D2025640A006D6B5F696E748B
:1005B000657276616C203D2025640A006D6B5F6476
:1005C000656C6179203D2025640A006D6B5F77685A
:1005D00065656C5F74696D655F746F5F6D617820D0
:1005E0003D2025640A006D6B5F776865656C5F6D03
:1005F00061785F7370656564203D2025640A006D35
:100600006B5F74696D655F746F5F6D6178203D200D
:1006100025640A006D6B5F6D61785F73706565645A
:10062000203D2025640A006D6B5F696E74657276EB
:10063000616C203D2025640A006D6B5F64656C6110
:1006400079203D2025640A000A00257500363A20ED
:10065000776865656C5F74696D655F746F5F6D6108
:10066000783A20000A00257500353A2077686565DC
:100670006C5F6D61785F73706565643A20000A0095
:10068000257500343A2074696D655F746F5F6D6124
:10069000783A20000A00257500333A206D61785FB2
:1006A00073706565643A20000A00257500323A20AF
:1006B000696E74657276616C286D73293A20000A40
:1006C00000257500313A2064656C6179282A313043
:1006D0006D73293A20000A092D2056616C756573E7
:1006E000202D0A004D3E004D25643E20003F007342
:1006F00065742064656661756C740A00433E200071
:1007000077686572652064656C74613A2063757200
:10071000736F723D25642C20776865656C3D256498
:100720000A53656520687474703A2F2F656E2E77B2
:10073000696B6970656469612E6F72672F77696B89
:10074000692F4D6F7573655F6B6579730A000A09D0
:100750002D204D6F7573656B6579202D0A455343C8
:100760002F713A09717569740A313A0964656C61CF
:1007700079282A31306D73290A323A09696E746515
:100780007276616C286D73290A333A096D61785F5E
:1007900073706565640A343A0974696D655F746FD6
:1007A0005F6D61780A353A09776865656C5F6D61E0
:1007B000785F73706565640A363A09776865656CB9
:1007C0005F74696D655F746F5F6D61780A0A703A76
:1007D000097072696E742076616C7565730A643A8B
:1007E000097365742064656661756C74730A75704D
:1007F0003A092B310A646F776E3A092D310A706716
:1008000075703A092B31300A7067646F776E3A0958
:100810002D31300A0A7370656564203D2064656C73
:100820007461202A206D61785F7370656564202A89
:100830002028726570656174202F2074696D655F72
:10084000746F5F6D6178290A003F004D3E200043C0
:100850003E20004C25640A000A092D20436F6E7368
:100860006F6C65202D0A4553432F713A09717569E4
:10087000740A6D3A096D6F7573656B65790A000AC4
:10088000092D204D61676963202D0A643A0964656A
:100890006275670A783A096465627567206D6174EC
:1008A0007269780A6B3A096465627567206B6579CD
:1008B000626F6172640A6D3A096465627567206DE2
:1008C0006F7573650A763A0976657273696F6E0A99
:1008D000733A097374617475730A633A09636F6ECE
:1008E000736F6C65206D6F64650A302D343A096C46
:1008F00061796572302D34284631302D4634290A0D
:10090000506175733A09626F6F746C6F61646572E0
:100910000A003F0074696D65725F7265616433320D
:1009200028293A202530346C580A006B6579626FAB
:100930006172645F69646C653A2025580A006B65D2
:1009400079626F6172645F70726F746F636F6C3A1B
:100950002025580A00686F73745F6B6579626F6158
:1009600072645F6C65647328293A2025580A000A6E
:10097000092D20537461747573202D0A0047434379
:100980003A20352E342E30204156522D4C494243C8
:100990003A20322E302E30204156525F4152434889
:1009A0003A20617672350A004F5054494F4E533AFF
:1009B000204C554641204D4F5553454B45592045F8
:1009C000585452414B455920434F4E534F4C4520AC
:1009D000434F4D4D414E44204B45594D41505F537F
:1009E000454354494F4E20343039360A0042554968
:1009F0004C443A20613336656666393220283135F9
:100A00003A34313A3332204A616E20323420323067
:100A10003231290A005649443A2030784645454447
:100A200028742E6D2E6B2E29205049443A203078A0
:100A30003041444228414442206B6579626F6172C3
:100A40006420636F6E766572746572292056455214
:100A50003A203078303130310A00444553433A204F
:100A6000636F6E7665727420414442206B657962D3
:100A70006F61726420746F205553420A000A092D79
:100A80002056657273696F6E202D0A000A6D6F75AE
:100A900073653A206F66660A000A6D6F7573653A72
:100AA000206F6E0A000A6B6579626F6172643A208A
:100AB0006F66660A000A6B6579626F6172643A203C
:100AC0006F6E0A000A6D61747269783A206F66660B
:100AD0000A000A6D61747269783A206F6E0A000A22
:100AE00064656275673A206F6E0A000A6465627514
:100AF000673A206F66660A000A0A626F6F746C6F4D
:100B0000616465722E2E2E2000433E2000001124C9
:100B10001FBECFEFDAE0DEBFCDBF04B603FE28C0B4
:100B20008091800390918103A0918203B09183030F
:100B30008730904BA740B04BD9F4109280031092AD
:100B40008103109282031092830314BE0FB6F894AF
:100B5000A895809160008861809360001092600089
:100B60000FBE1092010810920008E0E0F8E309952A
:100B700011E0A0E0B1E0EAE3F5E502C005900D92D6
:100B8000A235B107D9F723E0A2E5B1E001C01D927B
:100B9000A038B207E1F70E94340F0C949B2A0C9402
:100BA0000000FF93EF93E0915201F09153013097D1
:100BB00009F00995EF91FF910895FC01859180302E
:100BC00011F0EFDFFBCF0895FF27E0E230E247FFAF
:100BD0000CC0419597FF09C0EDE260957095809536
:100BE0009095611D711D811D911D27FF02C02195EA
:100BF00030E350E2AA27660F771F881F991FAA1FAC
:100C0000A41710F0A41B63955A95A9F7AA3008F011
:100C1000A95FA05DAF93F3956115710581059105FD
:100C200041F7ED3211F4EF93F395F21718F43F9377
:100C3000F395FBCF8F91B5DFFA95E1F70895E99130
:100C4000F9918591803021F0853219F0AADFF9CF32
:100C5000089520E0E89455915532C1F3503311F4D2
:100C6000689455915A3348F4505390F3220F022E52
:100C7000220F220F200D250FF4CF0EF4219589911C
:100C80009991533619F3533729F1533559F1BC0172
:100C900088279927E8945C3621F489919991689482
:100CA0005591543639F446EF7EF077FF0DC08FEF43
:100CB0009FEF0AC055374AE039F0583540E121F03E
:100CC000523642E009F00895FF93EF937DDFEF91F4
:100CD000FF91B7CFFF93EF93FC0181918030B9F37F
:100CE00060DFFBCFFF93EF9368DFF1CFDF93CF930C
:100CF000CDB7DEB72596A3DFCF91DF910895282FDA
:100D00002770E82FE695E695E695EF70F0E0E05A5B
:100D1000FE4F87FF0AC081E090E001C0880F2A954E
:100D2000EAF780959081892308C081E090E001C0B6
:100D3000880F2A95EAF79081892B808308950F9375
:100D40001F93CF93DF9389E892E09F938F930E9444
:100D500076060F900F90C0E0D0E004E712E063E069
:100D60008C2F0E94E60B009771F09F938F93DF9377
:100D7000CF931F930F930E9476060F900F900F90C2
:100D80000F900F900F902196C031D10541F7DF9160
:100D9000CF911F910F9108953F924F925F926F9262
:100DA0007F928F929F92AF92BF92CF92DF92EF92FB
:100DB000FF920F931F93CF93DF93CDB7DEB72897A2
:100DC0000FB6F894DEBF0FBECDBF80915901909150
:100DD0005A010E9433220C9708F484C20E941B22FD
:100DE00090935A0180935901809157019091580135
:100DF0000E943322893E934008F458C10E941B226E
:100E00009093580180935701EEEA4E2EE1E05E2E5A
:100E1000F7EB6F2EF1E07F2EA5EDCA2EA1E0DA2EC2
:100E2000BFECAB2EB1E0BB2E63E083E00E94E60B8B
:100E30008C01009709F43AC11F938F931F9283E0AE
:100E40008F938EE192E09F938F930E94760683E0CA
:100E50000E94570C412F4F602EEF63E083E00E9409
:100E6000450C8FE00E94570C63E08FE00E94E60B78
:100E70008C010F900F900F900F900F900F90009794
:100E800029F0982E74E6E72EF12C69C081E192E0FA
:100E90009F938F930E9476060F900F90C5CF8FE09F
:100EA0000E94570C24E0412F63E08FE00E94450C24
:100EB00063E08FE00E94E60B8C01982E31E08313F3
:100EC0000FC08FE00E94570C22E0412F63E08FE0BB
:100ED0000E94450C63E08FE00E94E60B8C01982E87
:100EE0001F930F931F928FE08F936CEF71E07F93AE
:100EF0006F930E9476060F900F900F900F900F90B7
:100F00000F9091E0991230C02CEE31E03F932F9377
:100F10000E947606F0921301E09212010F900F905A
:100F20008FE00E94570C412F407F4A602EEF63E014
:100F30008FE00E94450C8AE00E94570C63E08FE02E
:100F40000E94E60B8C01982E892B09F46DCF84E961
:100F500091E09F938F930E9476060F900F908FEFF2
:100F6000890D823088F49BCF62E096120DC08CED23
:100F700091E09F938F930E94760668EC70E07093E7
:100F8000130160931201CACF74E0971271C028E078
:100F9000AE014F5F5F4F61E08FE00E94610B8630D2
:100FA00050F02D813E8132272327322730931301C1
:100FB0002093120106C0F0921301E09212018823DF
:100FC000B9F1882E912C1F928F93DF92CF920E94BD
:100FD00076060F900F900F900F90312C832D032CDD
:100FE000000C990B881599059CF4E1E0F0E0EC0FFA
:100FF000FD1FE80FF91F80811F928F93BF92AF9260
:101000000E94760633940F900F900F900F90E6CFCA
:10101000809113018F93809112018F9385EC91E061
:101020009F938F930E9476060F900F900F900F90D2
:1010300089818B34C1F48A818D34A9F48B818C34FD
:1010400091F48C81813379F47F926F920E947606BD
:101050008FE00E94570C2EEF412F407F63E08FE01E
:101060000E94450C5BCF5F924F920E94760656CF4E
:1010700032E3931255CF64EA71E07F936F930E943D
:1010800076068FE00E94570C28E04AE051E062E0CB
:101090008FE00E940C0C8FE00E94570C28E042E089
:1010A00051E062E08FE00E940C0C38CF25E0AE01E9
:1010B0004F5F5F4F60E08AE00E94610B182F823023
:1010C00010F481E00DC18D811F928F938C811F924E
:1010D0008F938B811F928F938A811F928F93898127
:1010E0001F928F9386E592E09F938F930E947606DE
:1010F0000FB6F894DEBF0FBECDBF123049F4998110
:1011000096FB992790F98A8186FB882780F90AC087
:10111000FE01E10FF11D808186FB992790F982FB8A
:10112000882780F948EF58E81530E0F4212F012E88
:10113000000C330BE1E0F0E0EC0FFD1FE20FF31FBA
:10114000911102C0508301C04083882349F0E1E03F
:10115000F0E0EC0FFD1FE20FF31F208127602083DA
:101160001F5FE2CF2D8123FF02C080E001C080E835
:1011700027FF80644C8143FF806247FF80616B8161
:1011800063FF886067FF84603A8137FF826059811E
:1011900057FF816080935B01A62FA07778E0A79F1F
:1011A000D0011124942F907770E4979FF0011124BF
:1011B000EA2BFB2B5F77DF01A52BE22FE077F0E036
:1011C000FE2FEE27FF0FEA2BFB2B932F9F7730E0AC
:1011D000322F22273295330F307E292B677090E80B
:1011E000699FB0011124262B372B477050E0542FF4
:1011F0004427550F550F242B352B90915601A92FBD
:10120000092E000CBB0B2A9FA0012B9F500D3A9F6B
:10121000500D112441386FEF560714F441E85FEF89
:1012200051954195510941387FEF570714F441E832
:101230005FEF419540935C01EA9FB001EB9F700D19
:10124000FA9F700D112461385FEF750714F461E89F
:101250007FEF71956195710961385FEF750714F43F
:1012600061E87FEF619560935D01BF939F93FF936A
:10127000EF93E62F062E000CFF0BFF936F933F9327
:101280002F93242F042E000C330B3F934F931F9268
:101290008F9383E392E09F938F930E9476068BE572
:1012A00091E00E94141580915601482F082E000CE1
:1012B000550B0FB6F894DEBF0FBECDBF20911201C3
:1012C00030911301283C310518F428E030E002C0C9
:1012D00024E030E091E0421753070CF090E0890FD2
:1012E0008093560128960FB6F894DEBF0FBECDBF8F
:1012F000DF91CF911F910F91FF90EF90DF90CF90F2
:10130000BF90AF909F908F907F906F905F904F9025
:101310003F9008951F93CF93DF93C0910001D09128
:1013200001018FEF9FEF9093010180930001CF3F68
:101330008FEFD80721F580915401909155010E94BB
:1013400033220C9710F480E0B6C00E941B229093C9
:1013500055018093540182E00E94090CEC01892B15
:1013600009F447C0DF93CF938EE891E09F938F936A
:101370000E9476060F900F900F900F9002C020975A
:1013800011F3CF378FE7D80711F48FE705C0CF3FB0
:101390008FEFD80721F48FEF0E947F0628C08D2F92
:1013A0001C2FDF3F11F48C2F1FEF909170019923B8
:1013B00089F0982F9F77923319F480788A6004C05F
:1013C0009A3011F480788263982F9F779A3211F4C3
:1013D000807880670E947F061F3F49F0812F90E050
:1013E000982F88278F6F909301018093000181E0EF
:1013F00062C080917101882309F4A5CF87E00E9423
:10140000090CEC01892B09F49ECFDF93CF9386E87A
:1014100091E09F938F930E9476060F900F900F900C
:101420000F90CE018F7799278230910591F038F493
:10143000009761F0019799F4C078CA641AC08330AC
:10144000910551F08F379105A1F009C0C078C264B1
:1014500010C0C078C9640DC0C078C8640AC083E7F2
:1014600091E09F938F930E9476060F900F9081E1F9
:1014700022C08D2F99278F7799278130910561F0B0
:1014800040F08230910559F0039761F4D078D86428
:1014900078CFD078D26475CFD078DA6472CFD07834
:1014A000D9646FCF80E691E09F938F930E94760678
:1014B0000F900F9080E1DF91CF911F910895E82F59
:1014C000F0E0E05AFE4F80810895682F609582E039
:1014D0000C946E0C80916203816080936203569A33
:1014E0005E9A0E945D0B2FEF83ED90E321508040C8
:1014F0009040E1F700C000000E949F0685EB92E05B
:101500009F938F930E94760663E082E00E94E60B31
:1015100099270F900F908131910539F190F4873020
:10152000910519F138F49C0124503109223031051C
:1015300000F51BC089309105C1F08D309105C9F4CB
:1015400014C08D31910589F038F48431910569F02A
:101550008931910571F409C0843C910531F0873CD3
:10156000910519F0813C910521F421E0209370014F
:1015700002C01092700120917001211103C021E37B
:1015800031E002C02DE231E03F932F939F938F9380
:101590008DE992E09F938F930E94760663E087E047
:1015A0000E94E60B992721E00F900F900F900F906B
:1015B0000F900F908230910509F020E02093710187
:1015C000029741F481E992E09F938F930E947606FF
:1015D0000F900F9023E042E063E082E00E94450C10
:1015E000E0E6F1E0119221E0E037F207D9F70E943E
:1015F000BF140E94650A0E949F06569A5E9808953D
:10160000509A83E091E00197F1F700C000005098F4
:101610009AEB9A95F1F700C00895509A8AEB8A9553
:10162000F1F700C0509883E091E00197F1F700C016
:1016300000000895EF92FF920F931F93CF93DF93D3
:10164000C0E0D0E090E8E92EF12C082F10E0C701AF
:101650000C2E02C0959587950A94E2F7802391237A
:10166000892B19F00E940D0B02C00E94000B2196DD
:10167000C830D10561F7DF91CF911F910F91FF9095
:10168000EF900895509A83EF9BE00197F1F700C027
:1016900000000C940D0B489B06C023E02A95F1F73F
:1016A00000000197C1F70895489906C023E02A95E4
:1016B000F1F700000197C1F70895589850980895E0
:1016C0000895EF92FF920F931F93CF93DF93C82F4C
:1016D000162F7A01D22F80E0422F50E0282F082EBB
:1016E000000C330B2417350734F4F701E20FF31F16
:1016F00010828F5FF3CFF8940E94420B80E1C89F65
:1017000090011124812F8C60822B0E941A0B0E9461
:10171000000B84EF91E00E94540B892B19F485ECA7
:1017200092E01AC084EF91E00E944B0B892B19F4D0
:10173000789480E044C088E290E00E94540B892BAA
:1017400019F483EC92E008C084E690E00E944B0B11
:10175000892B51F481EC92E09F938F930E9476063F
:1017600078940F900F90E5CFC0E082E890E00E945F
:10177000540B8823F9F08C011127C8010E944B0BF0
:101780008823C1F09C2F9695969596959D1780F489
:10179000F701E90FF11D9081990F22E830E0201B3D
:1017A000310B081B1109201731070CF4916090834D
:1017B000CF5FD9F678948C2F869586958695DF91A4
:1017C000CF911F910F91FF90EF900895CF93DF93EA
:1017D000CDB7DEB728970FB6F894DEBF0FBECDBFEA
:1017E00028E0AE014F5F5F4F0E94610B823031F401
:1017F00089819A8198278927982702C080E090E004
:1018000028960FB6F894DEBF0FBECDBFDF91CF9103
:10181000089560E00C94E60BEF92FF921F93CF9334
:10182000DF93D82F162F7A01C22FF8940E94420B13
:1018300080E1D89F90011124812F8860822B0E9423
:101840001A0B0E94000B8FE193E00197F1F700C0A3
:1018500000000E940D0B10E0D0E0812F012E000C43
:10186000990B8C179D0744F4F701E80FF91F80814D
:101870000E941A0B1F5FF1CF0E94000B7894DF913A
:10188000CF911F91FF90EF900895CF93DF9300D0F9
:10189000CDB7DEB749832A8322E0AE014F5F5F4FA9
:1018A0000E940C0C0F900F90DF91CF910895CF9371
:1018B000C82FF8940E94420B20E1C29FC00111245E
:1018C00081600E941A0B0E94000B8FE193E0019748
:1018D000F1F700C000007894CF910895262F27706B
:1018E00040E062E00C94450C80917E020895CF9315
:1018F000DF9300D01F92CDB7DEB79C0180917703B4
:10190000843019F593E099833B832A839093E9000F
:101910008FEF9091E800815095FD06C095ED9A9566
:10192000F1F700008111F5CF8091E80085FF0DC02F
:1019300040E050E063E070E0CE0101960E94EA10C2
:101940008091E8008E778093E8000F900F900F90C1
:10195000DF91CF910895CF93DF9300D01F92CDB741
:10196000DEB720917703243031F522E029838058B7
:1019700091099B838A8383E08093E9008FEF9091A4
:10198000E800815095FD06C095ED9A95F1F70000AD
:101990008111F5CF8091E80085FF0DC040E050E057
:1019A00063E070E0CE0101960E94EA108091E800A9
:1019B0008E778093E8000F900F900F90DF91CF917A
:1019C0000895209177032430F1F422E02093E90078
:1019D0002FEF3091E800215035FD06C035ED3A95E6
:1019E000F1F700002111F5CF2091E80025FF0BC091
:1019F00040E050E065E070E00E94EA108091E8006D
:101A00008E778093E8000895CF93DF93209177033A
:101A1000243049F521E02093E90021E8215059F0D4
:101A20003091E80035FD07C0EFE3F1E03197F1F7C1
:101A300000C00000F3CF2091E80025FF14C0EC01A6
:101A400040E050E068E070E00E94EA108091E80019
:101A50008E778093E80088E0FE01A6E7B2E001906F
:101A60000D928A95E1F7DF91CF910895CF93C091C0
:101A70007401C1110BC00E942722643C794081058A
:101A8000910520F081E080937401C1E08C2FCF910B
:101A90000895FF920F931F93CF93DF93D82F0FB624
:101AA00007FE83C080917703843081F08091170115
:101AB00090E001962091190130E082239323209138
:101AC000180130E08217930709F0CDC00E94360D4F
:101AD000811110C08091170190E0019620911901A9
:101AE00030E0822393232091180130E0821793077E
:101AF00009F0B9C00E941B228C01C091E900CF708F
:101B00009091EC00892F817090FD80E8C82B84E0D3
:101B10008093E90085E0F82E8091EB0085FD42C0BE
:101B20008091EB0080FF3EC08091EE0087FF3AC0BD
:101B30008091180190911701981709F457C090915E
:101B4000E80095FF8EC0E0911501F0911601E80FB5
:101B5000F11D20818F5F90911901892380931801D5
:101B60002093F1008091E80085FDE2CF8091E800AC
:101B700080FFDECF8091E8008E778093E800F092BE
:101B80001401D6CF8091170190E0019620911901A0
:101B900030E0822393232091180130E082179307CD
:101BA00009F44CC0CF70C093E90040911701842F15
:101BB00090E001962091190130E082239323209137
:101BC000180130E08217930709F450C0E091150125
:101BD000F0911601E40FF11DD083809117018F5F02
:101BE0009091190189238093170140C08091E800EA
:101BF00085FF37C0D093F10021E03091F300809150
:101C0000F20090E0932B892B91F08091E80080FF07
:101C10000EC08091E80085FF03C01092F100F9CF5B
:101C20008091E8008E778093E800F09214012223DF
:101C300009F4A8CFCF70C093E90018C080911401B7
:101C4000882309F4AFCF0E941B229C0180179107C3
:101C500011F4890161CF9091140191509093140176
:101C6000F8CF20E0CACF40911701B0CF80E0DF91DC
:101C7000CF911F910F91FF9008958091760381116C
:101C800004C00E9456130C94B31308951092760367
:101C90000895089542E061EC81E00E94631042E003
:101CA00061EC82E00E94631042E061EC83E00E94FC
:101CB000631042E261EC84E00C946310809179033C
:101CC000833009F453C030F4813071F0823009F46C
:101CD0008CC008958A3009F478C08B3009F45EC056
:101CE000893009F09AC020C080917803813A09F0C8
:101CF00094C08091E800877F8093E80080917C0306
:101D000090917D03892B21F468E086E792E003C07F
:101D100060E080E090E070E00E9437118091E80080
:101D20008B778093E800089580917803813209F0E1
:101D300074C080917C0390917D03892B09F06DC064
:101D40008091E800877F8093E8008091E80082FD21
:101D500005C0809177038111F8CF5FC08091F100B9
:101D600080937E028091E8008B7753C08091780346
:101D7000813A09F052C080917C0390917D03892BB8
:101D800009F04BC08091E800877F8093E800809144
:101D9000E80080FFFCCF8091240136C08091780359
:101DA0008132D9F580917C0390917D03892BA9F52F
:101DB0008091E800877F8093E8000E9498108091CE
:101DC0007A03809324010C94CD178091780381329B
:101DD00021F58091E800877F8093E8000E949810A9
:101DE00080917B0380937F02089580917803813AEC
:101DF000A1F48091E800877F8093E8008091E8005B
:101E000080FFFCCF80917F028093F1008091E800F9
:101E10008E778093E8000C949810089580917E024C
:101E20008093750110927E020E9428160C94CD17A3
:101E30000C940E0F0E94A82180917503882329F02D
:101E40000E94D12181110C944D1008950E94E5212A
:101E50008091750180937E0208950C94260F089559
:101E60000C942F0F0C942F0FCF9384B7877F84BFD0
:101E70000FB6F894A8958091600088618093600007
:101E8000109260000FBE90E080E80FB6F894809347
:101E90006100909361000FBE89E49DE00E947B2168
:101EA0008AE191E00E94BA148BEE92E00E94DD0577
:101EB0000E94320F0E9479150E9456130E94B3139C
:101EC00078940E947B1580917703843029F00E94DA
:101ED0009F140E942F0FF7CF89ED92E00E94DD053D
:101EE0000E94300F87EC92E00E94DD05C4E08091F3
:101EF0007703853019F40E941A0FF9CF0E948115DB
:101F00002091E4003091E50080917201909173017D
:101F10002817390709F468C08091E4009091E50022
:101F200090937301809372010E94360D882309F407
:101F30005BC080917703843009F056C08091E9003E
:101F40008F702091EC00922F917020FD90E8892BEA
:101F5000C093E9009091EB0090FF43C09091EE0098
:101F600097FF3FC09091180120911701291709F19F
:101F70002091E80025FF1DC0E0911501F0911601A8
:101F8000E90FF11D30819F5F2091190192239093F9
:101F900018013093F1009091E80095FDE3CF909106
:101FA000E80090FFDFCF9091E8009E779093E800E3
:101FB000D9CF9091F3002091F20030E0392B232B00
:101FC00081F09091E80090FF0CC09091E80095FF9F
:101FD00003C01092F100F9CF9091E8009E779093A2
:101FE000E8008F708093E9000E949F1480CF292F12
:101FF000332723303105C9F060F42130310581F0F9
:102000002230310509F041C084E790E025E433E057
:1020100040C021323105E1F02232310531F135C0C5
:1020200082E190E029EB33E034C0992781309105BB
:1020300049F028F0029749F5E1E0F3E005C0E1E45A
:10204000F3E002C0E1E3F3E0849190E09F0121C05E
:1020500064307105D0F4660F771FFB01E05CFE4F22
:102060002081318189E090E014C06430710568F40A
:10207000FB01EE0FFF1FE85CFE4F20813181FB0169
:10208000EC5CFE4F808190E004C080E090E020E0B6
:1020900030E0FA0131832083089580E189BD82E137
:1020A00089BD09B400FEFDCF8091D8008F7D80935B
:1020B000D8008091E00082608093E0008091E00091
:1020C00081FDFCCF0895982F973068F59093E90033
:1020D000981739F07091EC002091ED005091F000CC
:1020E00003C0242F762F50E021FD02C09F5FECCF6C
:1020F0003091EB003E7F3093EB003091ED003D7F5F
:102100003093ED003091EB0031603093EB00709331
:10211000EC002093ED005093F0002091EE0027FD9D
:10212000E5CF80E008958F708093E90081E0089505
:102130008091780387FF11C08091E80082FD05C07F
:10214000809177038111F8CF11C08091E8008B77DF
:102150000BC080917703882349F08091E80080FFCD
:10216000F8CF8091E8008E778093E8000895209161
:10217000E4003091E50095E64091EC00842F8170F9
:1021800040FF23C08091E80080FD1DC0809177034F
:10219000882399F0853099F08091EB0085FD11C07E
:1021A0004091E4005091E5002417350729F3915040
:1021B00011F09A01E1CF84E0089582E0089583E070
:1021C000089581E0089580E008954091E80042FF7D
:1021D000DDCF0895CF92DF92EF92FF920F931F937E
:1021E000CF93DF93EC018B017A010E94B71081112C
:1021F00035C0E114F10439F0F70180819181081BA9
:10220000190BC80FD91FC12CD12C0115110529F1AB
:102210008091E80085FD18C08091E8008E7780935A
:10222000E8000E949F14E114F10449F0F701808155
:102230009181C80ED91ED182C08285E00FC00E9454
:10224000B710882311F30AC089918093F1000150DF
:102250001109FFEFCF1ADF0AD8CF80E0DF91CF91CD
:102260001F910F91FF90EF90DF90CF9008952091F4
:102270007E0330917F032617370748F061157105FB
:1022800039F42091E8002E772093E80001C0B901CD
:10229000FC0120E06115710579F1809177038823B5
:1022A000F1F18530F1F18091E80083FD3CC080912F
:1022B000E80082FD2EC08091E80080FFEBCF2091E6
:1022C000F3008091F20090E0922B6115710551F0BE
:1022D0008830910538F421912093F1006150710903
:1022E0000196F3CF21E0089709F020E08091E80003
:1022F0008E778093E800CECF2111CFCF0AC0809196
:102300007703882361F0853061F08091E80083FDD8
:102310000AC08091E80082FFF2CF80E0089582E059
:10232000089583E0089581E0089520917E0330911F
:102330007F032617370748F06115710539F420919E
:10234000E8002E772093E80001C0B901FC0120E0ED
:102350006115710591F180917703882309F440C0DC
:10236000853009F43FC08091E80083FD3DC0809135
:10237000E80082FD2FC08091E80080FFE9CF209126
:10238000F3008091F20090E0922B6115710559F0F5
:102390008830910540F424912093F10031966150EA
:1023A00071090196F2CF21E0089709F020E08091B1
:1023B000E8008E778093E800CBCF2111CCCF0AC004
:1023C00080917703882361F0853061F08091E80087
:1023D00083FD0AC08091E80082FFF2CF80E008957B
:1023E00082E0089583E0089581E008951F93CF93DC
:1023F000DF93CDB7DEB7AA970FB6F894DEBF0FBE56
:10240000CDBFE8E7F3E08091F100819323E0E0386D
:10241000F207C9F70E945E0E8091E80083FF2EC18B
:102420008091780390917903492F50E04A3051050B
:1024300008F024C1FA01EA5AFF4F0C94812A80382F
:1024400021F0823809F01AC108C08091740390917C
:102450007503992389F082600FC080917C038F708F
:10246000873008F00BC18093E9008091EB0085FB79
:10247000882780F91092E9009091E800977F909367
:10248000E8008093F1001092F100D1C0282F2D7F39
:1024900009F0F4C0882319F0823061F0EFC0809118
:1024A0007A03813009F0EAC0933009F080E080932C
:1024B00075032EC080917A0381112AC080917C031C
:1024C0008F702FEF280F263008F0D8C08093E900D6
:1024D0002091EB0020FF1CC0933021F48091EB0091
:1024E000806214C09091EB0090619093EB0021E02A
:1024F00030E0A90102C0440F551F8A95E2F74093CE
:10250000EA001092EA008091EB0088608093EB0073
:102510001092E9008091E800877F8093E8000E9494
:102520009810ACC08111AAC010917A031F778091D6
:10253000E3008078812B8093E3008091E800877F1F
:102540008093E8000E9498108091E80080FFFCCF03
:102550008091E30080688093E300111102C082E063
:1025600001C083E08093770389C08058823008F0EF
:1025700085C080917A0390917B038C3D53E0950751
:1025800079F583E08A838AE289834FB7F894DE0184
:10259000139620E03EE051E2E32FF0E05093570025
:1025A000E49120FF03C0E295EF703F5FEF708E2F44
:1025B00090E0EA3010F0C79601C0C0968D939D93CD
:1025C0002F5F243149F74FBF8091E800877F8093C8
:1025D000E8006AE270E0CE0101960E94371116C051
:1025E00060917C0370917D03AE014F5F5F4F0E944D
:1025F000F70FBC01892B09F441C09091E800977F47
:102600009093E80089819A810E9495118091E80059
:102610008B778093E80032C0803881F58091E800A4
:10262000877F8093E800809173038093F10080910D
:10263000E8008E7772CF811121C080917A0390914A
:102640007B0399270297D4F48091E800877F8093D9
:10265000E80080917A03809373030E949810809120
:102660007303811106C08091E30087FD02C081E001
:1026700001C084E0809377030E944A0E8091E800B5
:1026800083FF0AC08091E800877F8093E8008091F3
:10269000EB0080628093EB00AA960FB6F894DEBF41
:1026A0000FBECDBFDF91CF911F9108950E94C4133B
:1026B0000E94CC13E0EEF0E0808181608083E8ED41
:1026C000F0E080818F77808319BCA7EDB0E08C911A
:1026D0008E7F8C9380818F7E808310927603089505
:1026E0000F931F93CF93DF930E94C4130E94CC13C8
:1026F000C8EDD0E088818F7788838881806888835F
:1027000088818F7D888319BC1092770310927303A0
:10271000109275031092740300EE10E0F8018081AE
:102720008B7F808388818160888342E060E080E0E5
:102730000E946310E1EEF0E080818E7F8083E2EE04
:10274000F0E0808181608083808188608083F801EF
:1027500080818E7F8083888180618883DF91CF91A3
:102760001F910F910895E8EDF0E080818F7E8083C6
:10277000E7EDF0E080818160808384E082BF81E0CA
:10278000809376030C947013E8EDF0E080818E7FE7
:1027900080831092E20008951092DA001092E10016
:1027A00008951F920F920FB60F9211242F933F930B
:1027B0004F935F936F937F938F939F93AF93BF9349
:1027C000EF93FF938091E10082FF0BC08091E200C4
:1027D00082FF07C08091E1008B7F8093E1000E941F
:1027E0009E148091DA0080FF1FC08091D80080FF86
:1027F0001BC08091DA008E7F8093DA008091D9002F
:1028000080FF0DC080E189BD82E189BD09B400FE71
:10281000FDCF81E0809377030E943D0E05C019BC77
:10282000109277030E94460E8091E10080FF19C04C
:102830008091E20080FF15C08091E2008E7F80933E
:10284000E2008091E20080618093E2008091D800F4
:1028500080628093D80019BC85E0809377030E9442
:10286000180F8091E10084FF30C08091E20084FF66
:102870002CC080E189BD82E189BD09B400FEFDCF95
:102880008091D8008F7D8093D8008091E1008F7E69
:102890008093E1008091E2008F7E8093E20080913E
:1028A000E20081608093E20080917303882311F03D
:1028B00084E007C08091E30087FD02C081E001C091
:1028C00083E0809377030E942D0F8091E10083FFC6
:1028D00024C08091E20083FF20C08091E100877FC7
:1028E0008093E10082E080937703109273038091DC
:1028F000E1008E7F8093E1008091E2008E7F8093E3
:10290000E2008091E20080618093E20042E060E0BA
:1029100080E00E9463100E94490EFF91EF91BF91E9
:10292000AF919F918F917F916F915F914F913F9167
:102930002F910F900FBE0F901F9018950895CF9371
:10294000809177038823A1F0C091E900CF70909126
:10295000EC00892F817090FD80E8C82B1092E9006F
:102960008091E80083FD0E94F611CF70C093E900CA
:10297000CF91089590938502809384020895E09109
:102980008402F0918502309721F00190F081E02DD2
:10299000099480E00895EF92FF920F931F93CF93D5
:1029A000DF93E0918402F09185023097B1F18C01C0
:1029B0000280F381E02D09958091620382FF2DC092
:1029C00080FF04C086ED94E00E94DD05E80118E078
:1029D00080EDE82E84E0F82E8091620380FF0BC02A
:1029E00088811F928F93FF92EF920E9476060F903C
:1029F0000F900F900F90115021961111EDCF8091F3
:102A0000620380FF0AC08EEC94E0DF91CF911F91AA
:102A10000F91FF90EF900C94DD05DF91CF911F9106
:102A20000F91FF90EF900895E0918402F09185025C
:102A3000309721F00480F581E02D09940895CF931B
:102A4000DF9320918202309183022817390709F120
:102A50009093830280938202E0918402F091850238
:102A60003097B9F0EC010680F781E02D099580914F
:102A7000620382FF0EC080FF0CC0DF93CF9380EC17
:102A800094E09F938F930E9476060F900F900F9083
:102A90000F90DF91CF910895CF93DF932091800223
:102AA000309181022817390709F1909381028093B0
:102AB0008002E0918402F09185023097B9F0EC0138
:102AC0000084F185E02D09958091620382FF0EC09C
:102AD00080FF0CC0DF93CF9380EB94E09F938F93A4
:102AE0000E9476060F900F900F900F90DF91CF917C
:102AF00008950C9429160E9412220E946A0A0C94CE
:102B0000600BBF92CF92DF92EF92FF920F931F93D1
:102B1000CF93DF9300D000D01F92CDB7DEB70E94D5
:102B20008A0907E812E0F12C8F2D0E945F0AB82E67
:102B3000F801C080C82639F4F3940F5F1F4FF0E10D
:102B4000FF12F2CF30C08091620381FD0E943E16D9
:102B5000D12CEE24E3948C2D8E21F9F0D982FA82C7
:102B600091E08B2D8E2109F490E09B830E941B2223
:102B70008160782F9D838C8349815A816B818D81FF
:102B80000E94741649815A816B817C818D810E94DB
:102B90009321F80180818E258083D394EE0CF8E098
:102BA000DF12D9CFC9CF8FEF89838A831B820E941E
:102BB0001B228160782F9D838C8349815A816B8190
:102BC0008D810E9474160E9492210E94BF240E944F
:102BD000CC060E94BF1490918602891741F10E9491
:102BE000BF14809386029091620392FF0EC090FF03
:102BF0000CC01F928F9381EE94E09F938F930E945D
:102C000076060F900F900F900F90809186020F9094
:102C10000F900F900F900F90DF91CF911F910F9118
:102C2000FF90EF90DF90CF90BF900C94A4210F9075
:102C30000F900F900F900F90DF91CF911F910F91F8
:102C4000FF90EF90DF90CF90BF9008950C94650AAD
:102C500008950895CF93C62F0E945F0A21E030E0C7
:102C600002C0220F331FCA95E2F790E028233923D0
:102C700081E0232B09F480E0CF910895EF92FF9239
:102C80000F931F93CF93DF9387EF94E00E94DD05AE
:102C9000C0E0D0E083E3E82E81E0F82E0CEE14E0F3
:102CA0008C2F0E945F0A0E948021FF92EF921F9258
:102CB0008F93DF93CF931F930F930E9476062196F5
:102CC0008DB79EB708960FB6F8949EBF0FBE8DBF06
:102CD000C031D10529F7DF91CF911F910F91FF905E
:102CE000EF90089508950895CF93DF93CDB7DEB7A1
:102CF0002B970FB6F894DEBF0FBECDBF942F4F8336
:102D0000252F588769877A878B874A855B85452B6E
:102D100031F02F3F31F481E09F3F19F403C081E08F
:102D200001C080E080FD07C04F81588569857A85A4
:102D30008B850E949321DE01119686E0FD011192A0
:102D40008A95E9F785E0FE01379601900D928A9504
:102D5000E1F749815A816B817C818D819E810E943E
:102D6000F51D2B960FB6F894DEBF0FBECDBFDF91D9
:102D7000CF910895CF93DF93882309F48FC0C82F94
:102D80008EE78C0F833018F5C23829F0C33831F044
:102D9000C4E0D7E405C0C2E0D9E302C0C1E0D3E596
:102DA0000E94BF148C2309F079C08D2F0E94DD2072
:102DB0000E9455212FEF81EE94E0215080409040F9
:102DC000E1F700C000008D2F0E94FA2010C08CEFA8
:102DD0008C0F813A20F080E58C0F8E3260F48C2FBE
:102DE0000E94E92781115AC08C2F0E94DD20DF91BB
:102DF000CF910C94552180E28C0F883048F4C77035
:102E000081E001C0880FCA95EAF70E941B21EFCF2D
:102E10008BE58C0F833080F4C53A29F0C63A31F047
:102E200083E890E005C081E890E002C082E890E08D
:102E3000DF91CF910C941F1588E58C0F873170F5C9
:102E4000C83A89F0C93A91F0CA3A99F0CB3AA1F060
:102E5000CC3AA9F0CD3AB1F0CE3AB9F0CF3AC1F0C0
:102E600080E090E017C082EE90E014C089EE90E020
:102E700011C08AEE90E00EC085EB90E00BC086EBAF
:102E800090E008C083EB90E005C084EB90E002C0C6
:102E900087EB90E0DF91CF910C944C15DF91CF91AF
:102EA0000895CF93DF93882309F454C09EE7980FC9
:102EB000933008F5823829F0833831F0C4E0D7E444
:102EC00005C0C2E0D9E302C0C1E0D3E50E94BF144F
:102ED0008C2309F43FC08D2F0E94DD200E945521D4
:102EE0002FEF81EE94E0215080409040E1F700C048
:102EF00000008D2F08C09CEF980F913A20F090E5CC
:102F0000980F9E3218F40E94FA200DC090E2980F9C
:102F1000983068F4877091E001C0990F8A95EAF7BC
:102F2000892F0E942121DF91CF910C9455219BE59F
:102F3000980F933030F480E090E0DF91CF910C94C3
:102F40001F15885A873130F480E090E0DF91CF91EF
:102F50000C944C15DF91CF910895882321F00E94A5
:102F60001B210C9455210895882321F00E942121D2
:102F70000C94552108950E943B210E940A210E9431
:102F800055210E9464250E94322480E090E00E9436
:102F90001F1580E090E00C944C150E942B210C949E
:102FA000BB17CF92DF92EF92FF920F931F93CF93B5
:102FB000DF9300D000D01F92CDB7DEB76C010E9426
:102FC000A621811118C385E0F601DE01119601905A
:102FD0000D928A95E1F7F601408151812381348178
:102FE0002115310531F05F3F31F481E04F3F19F495
:102FF00003C081E001C080E080FDFDC2F601F280E7
:10300000E580E2948FE0E82249835A83FB82722FA5
:103010003D832C836F2D8D810E9459208C010E944D
:1030200058200E94481FE12FE295EF708E2F90E00C
:10303000FC01E05AFF4F0C94812A812F807F1F7082
:10304000882311F01295107FFF20B9F0112329F089
:10305000812F0E942E210E945521802F0F900F90CA
:103060000F900F900F90DF91CF911F910F91FF90D4
:10307000EF90DF90CF900C94BA16802F0E945117DA
:10308000112309F4B8C2812F0E9434210F900F90B0
:103090000F900F900F90DF91CF911F910F91FF90A4
:1030A000EF90DF90CF900C945521812F807F1F707F
:1030B000803211F01295107F002319F0013009F1D0
:1030C0002BC0FF20A9F0EE2059F1F1E0812FEF1283
:1030D00028C00F900F900F900F900F90DF91CF911D
:1030E0001F910F91FF90EF90DF90CF900C943E21B5
:1030F000EE2021F021E0E21609F47DC20E94412178
:103100004DC0FF20E9F085E08E1508F474C20E94DE
:103110001821812329F042C0FF20F1F1E11015C0F0
:10312000812F0F900F900F900F900F90DF91CF9104
:103130001F910F91FF90EF90DF90CF900C94AD17FF
:1031400094E09E1508F457C229C0F601858180FFDE
:1031500013C08F708583E4CF003F09F489C108F064
:1031600055C180E4800F803208F459C1FF2009F472
:10317000EAC1EE2009F49AC1802F0E94BA160933E1
:1031800009F0DAC1FFEF21EE84E0F15020408040E9
:10319000E1F700C000002FC2E110D7C1812F59C153
:1031A000812F86958695837019F08130B9F023C2FE
:1031B000FF2019F0C801937002C080E090E00F90EA
:1031C0000F900F900F900F90DF91CF911F910F9163
:1031D000FF90EF90DF90CF900C941F15FF2019F017
:1031E000C801937002C080E090E00F900F900F90A4
:1031F0000F900F90DF91CF911F910F91FF90EF9063
:10320000DF90CF900C944C15802FFF2019F00E9476
:10321000452302C00E94AD230F900F900F900F9096
:103220000F90DF91CF911F910F91FF90EF90DF9062
:10323000CF900C943224812F837009F070C0F1106C
:10324000DAC1202F229526952770220F220F602F9A
:103250006F70862F90E0A0E0B0E06C017D01022E3F
:1032600004C0CC0CDD1CEE1CFF1C0A94D2F704FF3A
:1032700012C08FE090E0A0E0B0E004C0880F991F7A
:10328000AA1FBB1F2A95D2F7BC01CD01609570958E
:103290008095909503C060E070E0CB01169516957F
:1032A00013701230B1F040F56C297D298E299F29C9
:1032B000113031F10F900F900F900F900F90DF9120
:1032C000CF911F910F91FF90EF90DF90CF900C94D2
:1032D0006D1F6C297D298E299F290F900F900F90CB
:1032E0000F900F90DF91CF911F910F91FF90EF9072
:1032F000DF90CF900C94871F0E946D1FC701B6010D
:103300000F900F900F900F900F90DF91CF911F9122
:103310000F91FF90EF90DF90CF900C94531FFF2000
:1033200019F0812F817001C08695882309F463C14B
:10333000202F229526952770220F220F602F6F7065
:10334000862F90E0A0E0B0E06C017D01022E04C069
:10335000CC0CDD1CEE1CFF1C0A94D2F704FF12C03B
:103360008FE090E0A0E0B0E004C0880F991FAA1F92
:10337000BB1F2A95D2F7BC01CD0160957095809551
:10338000909503C060E070E0CB0116951695137020
:103390001230B1F040F56C297D298E299F2911301A
:1033A00031F10F900F900F900F900F90DF91CF9110
:1033B0001F910F91FF90EF90DF90CF900C943420ED
:1033C0006C297D298E299F290F900F900F900F90C7
:1033D0000F90DF91CF911F910F91FF90EF90DF90B1
:1033E000CF900C9446200E943420C701B6010F9064
:1033F0000F900F900F900F90DF91CF911F910F9131
:10340000FF90EF90DF90CF900C942220023F09F4C0
:103410005EC008F449C0033F09F46CC0A7CE902FEA
:103420009071E92E812F8F71FF2051F00E94BB1FF8
:10343000802FEE2019F08295807F73CE8F7071CE31
:103440000E94DC1F802FEE2019F08295807F01C042
:103450008F700F900F900F900F900F90DF91CF9182
:103460001F910F91FF90EF90DF90CF900C94B417C5
:10347000FF20A9F0E4E0EE1508F4BDC0812F8F71A4
:103480000F900F900F900F900F90DF91CF911F91A1
:103490000F91FF90EF90DF90CF900C940120F5E01A
:1034A000FE1508F4A8C0EACFFF2099F0812F8F7194
:1034B0000F900F900F900F900F90DF91CF911F9171
:1034C0000F91FF90EF90DF90CF900C94BB1FFF20E7
:1034D00069F3812F8F710F900F900F900F900F90C5
:1034E000DF91CF911F910F91FF90EF90DF90CF90E0
:1034F0000C94DC1FFF2089F0812F8F710F900F90AB
:103500000F900F900F90DF91CF911F910F91FF902F
:10351000EF90DF90CF900C94A61F0F900F900F901C
:103520000F900F90DF91CF911F910F91FF90EF902F
:10353000DF90CF900C94A11F033509F423CE0734FC
:1035400009F059C01FCEEE2021F2802F0F900F906E
:103550000F900F900F90DF91CF911F910F91FF90DF
:10356000EF90DF90CF900C945117412F4F70602F48
:10357000C6010E94BF220F900F900F900F900F90E6
:10358000DF91CF911F910F91FF90EF90DF90CF903F
:103590000C94A31E01112FC0FF2069F10E94CD17CA
:1035A0002FEF80E792E0215080409040E1F700C08B
:1035B00000000F900F900F900F900F90DF91CF9120
:1035C0001F910F91FF90EF90DF90CF900C946822A5
:1035D000412F4F70602FC6010F900F900F900F90EA
:1035E0000F90DF91CF911F910F91FF90EF90DF909F
:1035F000CF900C94C2220F900F900F900F900F90CD
:10360000DF91CF911F910F91FF90EF90DF90CF90BE
:1036100008951F93CF93DF9300D000D01F92CDB7B2
:10362000DEB7942F4983252F5A836B837C838D8348
:103630004C815D81452B31F02F3F31F481E09F3F7C
:1036400019F403C081E001C080E0182F117080FDE3
:1036500031C049815A816B817C818D810E945920C2
:10366000292F22952F702C3030F42A30A0F42250CC
:10367000223030F022C02C30C9F02F30B9F01DC0FC
:10368000853A28F48430C0F4823028F415C090E2E2
:10369000980F983088F0883E30F4803E68F484506B
:1036A000813A58F409C0803F41F406C093FB1127CA
:1036B00010F903C010E001C011E0812F0F900F90AE
:1036C0000F900F900F90DF91CF911F910895CF939E
:1036D000DF9300D000D01F92CDB7DEB70F900F90D0
:1036E0000F900F900F90DF91CF910895CF93DF93BC
:1036F00000D000D000D0CDB7DEB726960FB6F89434
:10370000DEBF0FBECDBFDF91CF9108951F93CF9342
:10371000DF93C091970216E080919802C81799F044
:10372000D0E01C9FF0011D9FF00D1124E756FD4FC6
:103730004081518162817381848195810E94761BD1
:103740002196C770E9CFDF91CF911F9108954091E5
:10375000C9025091CA026091CB027091CC02809153
:10376000CD029091CE020C94761B0F931F93CF93B2
:10377000DF938091CE0282958F7009F05DC08091B9
:10378000CB02882309F458C08091970210919802C7
:103790006091C9027091CA02C091CC02D091CD0251
:1037A00091E06F3F09F090E0292F06E0811709F4BE
:1037B00043C0209721F07F3F21F030E003C031E08B
:1037C00001C0322F90E030FD34C0089FF001099F06
:1037D000F00D1124DF01A756BD4F11963C911197B2
:1037E000371327C03C91361324C012963C91129790
:1037F00031111FC013964D915C9114974C1B5D0BBA
:10380000483C5105B0F48091CE028F708061809366
:10381000CE02E256FD4F80818F708061808389ECFB
:1038200092E00E94D117DF91CF911F910F910C94DC
:10383000861B01968770BACFDF91CF911F910F91B0
:1038400008959F92AF92BF92CF92DF92EF92FF9234
:103850000F931F93CF93DF93CDB7DEB761970FB66A
:10386000F894DEBF0FBECDBF8C0185E0F801DE010C
:103870001D9601900D928A95E1F7F80140815181E2
:10388000F280C380D4809091C9026091CA022091D5
:10389000CC023091CD022115310531F06F3F31F46A
:1038A00081E09F3F19F403C081E001C080E0F82F60
:1038B000F1709F2E80FD52C189ECA82E82E0B82EB7
:1038C000E090CB02F601E21BF30BEE2009F4E8C016
:1038D0008091CE02E83CF10508F0A4C0282F207F9B
:1038E00009F053C0561313C0491311C0EF2CF11047
:1038F0000EC08F7080618093CE020E94A71BC5010D
:103900000E94D1178091CE02F80185835BC1C1145A
:10391000D10431F05F3F31F481E04F3F19F403C02F
:1039200081E001C080E080FD03C081E08F2502C0FE
:1039300080E090E0F82FF170EF2E80FF1CC08091A6
:1039400097022091980236E0821709F418C190E09E
:10395000389FF001399FF00D1124E756FD4F61812A
:10396000561306C06081461303C06281F61203C07D
:1039700001968770E9CFEF2CFF2009F423C18091D5
:10398000CE0281608093CE0262C0561306C04913F6
:1039900004C0F11002C0F801A7C04D875E87FF8602
:1039A0007C2DD98AC88A6F2D89890E94091B88239A
:1039B00099F1FF2089F12091CE02822F82958F709C
:1039C00090E0029774F08091C9029091CA029887A2
:1039D0008F831986DB86CA862C87CE0107960E94C4
:1039E000D11786E0F801A9ECB2E001900D928A951A
:1039F000E1F70E94B51B0E94A71B11C0561749F1A1
:103A00004D875E87FF867C2DD98AC88A6F2D89896C
:103A10000E94091B81112CC0C8010E94D117EE24FD
:103A2000E394D0C0282F207F49F77C2DD98AC88AFB
:103A30006F2D89890E94671B89EC92E00E94D11743
:103A400086E0F50111928A95E9F70E94A71BE12C07
:103A5000B9C04913D5CFF110D3CFF8018583C80180
:103A60000E94D11786E0F50111928A95E9F7AAC064
:103A7000FF2091F22091CE02822F82958F7090E0EC
:103A800002970CF4AECF8091C9029091CA029A833A
:103A900089831B82DD82CC822E83CE0101969FCF4B
:103AA000E83CF10508F04BC0EF2CFF2009F4B4CF3F
:103AB000561330C049132EC02091CE0220FD21C0E4
:103AC000822F82958F70482F50E041155105C9F023
:103AD000F80125834F30510541F08F5F982F929563
:103AE000907F822F8F70892B8583C8010E94D11708
:103AF00086E0F801A9ECB2E001900D928A95E1F719
:103B00002AC086E0F801A9ECB2E001900D928A95F6
:103B1000E1F758C04D875E87FF867C2DD98AC88A19
:103B20006F2D89890E94091B81115BCF8091CE0284
:103B300081608093CE02C8010E94D11743C07C2DC2
:103B4000D98AC88A6F2D89890E94671B86E0F50192
:103B500011928A95E9F70E94A71B34C0FF2009F44F
:103B60005BCF4D875E87FF867C2DD98AC88A6F2DF3
:103B700089890E94091B882309F44ECF32CF7C2DFE
:103B8000D98AC88A6F2D89890E945920292F2295A8
:103B90002F70223028F49F7039F0811105C00BC0BE
:103BA000243028F49F7049F4805E883020F0C801EA
:103BB0000E94D1179E2CE92C05C0F8019581907FB9
:103BC00099F7F9CF8E2D61960FB6F894DEBF0FBE30
:103BD000CDBFDF91CF911F910F91FF90EF90DF90BC
:103BE000CF90BF90AF909F9008951F93CF93DF9396
:103BF000CDB7DEB72C970FB6F894DEBF0FBECDBFA2
:103C00004F83588769877A878B879C87CE01079671
:103C10000E94211C8823D1F09F8188852A853B85BD
:103C2000232B31F08F3F31F481E09F3F19F403C023
:103C300081E001C080E080FD47C04F8158856985E3
:103C40007A858B859C850E94761B3EC086E0FE01AE
:103C50003796DE01119601900D928A95E1F7FF816A
:103C6000E8856A857B856115710531F0EF3F31F498
:103C700081E0FF3F19F403C081E001C080E080FDD6
:103C800023C02091980230E0C901019687709927DE
:103C90004091970250E084179507F1F1F983EA8388
:103CA0007D836C8396E0929FD001939FB00D112489
:103CB000A756BD4FFE01319601900D929A95E1F7FE
:103CC000809398020E94861B16E080919702909143
:103CD0009802891771F1189FC001112487569D4FD2
:103CE0000E94211C882329F1E09197021E9FF00178
:103CF0001124E756FD4F4081518162817381848197
:103D000095810E94761B8091970290E001968770C2
:103D1000992780939702D9CF0E94CD1710929802CD
:103D200010929702E9ECF2E086E0DF011D928A959D
:103D3000E9F72C960FB6F894DEBF0FBECDBFDF912A
:103D4000CF911F910895DF92EF92FF920F931F93EF
:103D5000CF93DF93FC01892B09F488C0E12CF12C6F
:103D6000DD24D394EF0121968491853709F460C056
:103D700058F4843708F04EC0843008F068C08130B1
:103D8000D1F0823071F172C0883709F45BC050F411
:103D9000863709F453C0873709F068C08E2D0E941A
:103DA000282152C09CE7980F903708F05FC08F77AA
:103DB0000E9451174EC08F010E5F1F4FFE0184916C
:103DC00090E2980F983050F48770FD2D01C0FF0FDE
:103DD0008A95EAF78F2F0E942E2115C00E94BA16ED
:103DE00014C08F010E5F1F4FFE01849190E2980F67
:103DF000983068F48770FD2D01C0FF0F8A95EAF7AF
:103E00008F2F0E9434210E945521E80122C00E9478
:103E10005117FBCFCF010296FE01C491CC2361F074
:103E2000EFE9FFE03197F1F700C00000C150F6CF95
:103E3000CF010296FE01F490EC010BC00E94182104
:103E4000E82E07C00E942B210E94552102C00E942B
:103E5000BA168F2D882341F0EFE9FFE03197F1F793
:103E600000C000008150F6CFFE017CCFDF91CF91E2
:103E70001F910F91FF90EF90DF90089560934F0393
:103E80007093500380935103909352030C94A32199
:103E90000895609353037093540380935503909354
:103EA00056030C94A2210F931F930091530310917A
:103EB00054032091550330915603602B712B822BB4
:103EC000932B609353037093540380935503909303
:103ED00056031F910F910C94A2210F931F930091F1
:103EE00053031091540320915503309156036023DE
:103EF000712382239323609353037093540380931D
:103F00005503909356031F910F910C94A2210F9388
:103F10001F93009153031091540320915503309146
:103F2000560360277127822793276093530370936A
:103F3000540380935503909356031F910F910C9453
:103F4000A22160E070E0CB010C943E1F0F931F9301
:103F500041E050E060E070E08A019B0104C0000F86
:103F6000111F221F331F8A95D2F7C901B8011F9173
:103F70000F910C943E1F0F931F9341E050E060E0BF
:103F800070E004C0440F551F661F771F8A95D2F753
:103F900080914F0390915003A0915103B09152032F
:103FA0008A019B01082B192B2A2B3B2BC901B80135
:103FB0001F910F910C943E1F0F931F9341E050E00F
:103FC00060E070E004C0440F551F661F771F8A959C
:103FD000D2F7409550956095709580914F039091E0
:103FE0005003A0915103B09152038A019B01082311
:103FF00019232A233B23C901B8011F910F910C9467
:104000003E1F0F931F9341E050E060E070E004C05A
:10401000440F551F661F771F8A95D2F780914F0373
:1040200090915003A0915103B09152038A019B01DA
:10403000082719272A273B27C901B8011F910F918B
:104040000C943E1F0F931F9300914F031091500348
:104050002091510330915203602B712B822B932BB3
:104060001F910F910C943E1F0F931F9300914F03CC
:10407000109150032091510330915203602371231A
:10408000822393231F910F910C943E1F0F931F9334
:1040900000914F031091500320915103309152032E
:1040A00060277127822793271F910F910C943E1F41
:1040B00008958F929F92AF92BF92DF92EF92FF92FC
:1040C0000F931F93CF93DF9300D000D01F92CDB7F3
:1040D000DEB76B837C838D838A018C819D81892BE4
:1040E00031F01F3F31F481E04F3F19F403C081E00C
:1040F00001C080E080FF03C080E090E04DC08B8174
:104100008823D1F180904F0390905003A0905103E9
:10411000B09052038091530390915403A0915503A2
:10412000B0915603882A992AAA2ABB2A8FE1E82E41
:10413000F12CD501C4010E2C04C0B695A795979516
:1041400087950A94D2F780FD06C081E0E81AF1084D
:1041500080F7D12C07C0DE2CB8018E2D0E9497224B
:10416000019799F388E0189FF0011124E153FD4F66
:10417000E00FF11DD08209C088E0189FF0011124E2
:10418000E153FD4FE00FF11DD08009831A8369814F
:104190007A818D2D0E9497220F900F900F900F9093
:1041A0000F90DF91CF911F910F91FF90EF90DF90D3
:1041B000BF90AF909F908F900895209125013091EE
:1041C0002601F90132969FEF40E05191851789F061
:1041D0009F3F19F4511101C0942F4F5F4630A9F74A
:1041E0009F3F39F0F901E90FF11D97FDFA958283A0
:1041F00008950895E0912501F09126019F012A5F1D
:104200003F4F9281891301C012823196E217F30762
:10421000C1F7089581E090E0E0912501F091260139
:10422000E80FF91F1082019688309105A9F70895CB
:1042300080916103089590916103892B80936103BC
:104240000895809590916103892380936103089577
:104250008093610308951092610308959091600323
:10426000892B809360030895809590916003892342
:10427000809360030895109260030895809357031C
:104280000895109257030895809125019091260179
:10429000FC0131969C01285F3F4F80E09191911184
:1042A0008F5FE217F307D1F70895E0912501F091B0
:1042B0002601809161038083E0912501F091260120
:1042C000908180916003892B80838091570388239C
:1042D00061F0E0912501F09126019081892B808386
:1042E0000E944421811110925703809125019091E1
:1042F00026010C94CB14909353018093520108959E
:104300008295982F937344E0949F900111248C7CA4
:1043100086958695282B822F8575880F2A7A269573
:10432000822B08950895CF93DF9300D000D01F9281
:10433000CDB7DEB70F900F900F900F900F90DF91D9
:10434000CF910895089508950C94261680E008955D
:1043500080917703843021F11092630320E488E197
:1043600090E00FB6F894A895809360000FBE20935C
:10437000600083B7817F846083BF83B7816083BF20
:104380007894889583B78E7F83BF0FB6F894A895ED
:1043900080916000886180936000109260000FBE81
:1043A0000895CF930E9472160E948A090E94731684
:1043B000C0E08C2F0E945F0A811104C0CF5FC03122
:1043C000C1F701C081E0CF9108950E9428160C9496
:1043D000CD171F920F920FB60F9211248F939F93B8
:1043E000AF93BF9380916303811113C080916403E5
:1043F00090916503A0916603B09167034196A11D5A
:10440000B11D8093640390936503A0936603B093FA
:104410006703BF91AF919F918F910F900FBE0F9047
:104420001F90189582E084BD93E095BD9AEF97BDEB
:1044300080936E0008952FB7F89480916403909153
:104440006503A0916603B09167032FBF08952FB74E
:10445000F894609164037091650380916603909174
:1044600067032FBF08959C014FB7F89480916403B0
:1044700090916503A0916603B09167034FBF821BC3
:10448000930B089578941F920F920FB60F921124F8
:104490008F939F93AF93BF93809164039091650333
:1044A000A0916603B09167030196A11DB11D809391
:1044B000640390936503A0936603B0936703BF9171
:1044C000AF919F918F910F900FBE0F901F901895F5
:1044D0000E945613F89487E797E79093010880931A
:1044E000000887E090EBDC018093800390938103C8
:1044F000A0938203B09383039CE088E10FB6F89405
:10450000A895809360000FBE90936000FFCFE82FC6
:10451000F0E088E0989FE00DF11D1124E052FF4F7C
:104520008491982F92959F708F7097700895CF9374
:10453000C82FCB010E94872240E1949F9001112453
:10454000282B203831051CF080E090E016C09770D1
:10455000E92FF0E098E0C99FE00DF11D112494E0EF
:10456000EE0FFF1F9A95E1F78F70E80FF11DEE0F28
:10457000FF1FE050F84985919491CF91089580E014
:1045800090E00895089580916A0380FF0BC06091C8
:104590002A0185E0689FB00111247595679575958E
:1045A00067952BC081FF09C060912A0185E0689F53
:1045B000B00111247595679520C082FF07C06091F6
:1045C0002A0185E0689FB001112417C090916B0308
:1045D0009923D1F060912901961788F720912A013B
:1045E00085E0289F90011124929FA001939F500D78
:1045F000112470E0CA010E946D2A6038710540F4F0
:104600006115710519F406C065E070E0862F089504
:104610008FE7089581E0089580916A0380FF08C0C4
:104620006091280170E0759567957595679521C033
:1046300081FF06C06091280170E07595679519C0EB
:1046400082FF04C06091280170E010C090916B035C
:10465000992399F0609127019617A0F7809128017E
:10466000899FC001112470E00E946D2A6038710595
:1046700040F46115710519F406C061E070E0862F01
:1046800008958FE7089581E00895803F21F40E9406
:10469000C322819504C0813F29F40E94C3228093E4
:1046A0006E030895823F21F40E94C322819504C0C5
:1046B000833F29F40E94C32280936D030895893FAC
:1046C00019F40E940C2305C08A3F31F40E940C2388
:1046D000819580936F0308958B3F21F40E940C23F2
:1046E000819504C08C3F29F40E940C2380937003B1
:1046F0000895843F21F480916C03816017C0853F49
:1047000021F480916C03826011C0863F21F4809176
:104710006C0384600BC0873F21F480916C03886038
:1047200005C0883F31F480916C03806180936C03F5
:1047300008958D3F21F480916A0381600BC08E3F04
:1047400021F480916A03826005C08F3F29F4809133
:104750006A03846080936A030895803F39F48091EE
:104760006E0387FF6CC010926E0369C0813F29F40D
:1047700080916E031816BCF362C090916D03823F66
:1047800029F497FF5CC010926D0359C0833F19F460
:104790001916CCF354C0893F41F480916F03181669
:1047A0000CF04DC010926F034AC08A3F29F48091EB
:1047B0006F0387FF44C0F6CF8B3F39F480917003BD
:1047C00087FF3DC0109270033AC08C3F29F480915E
:1047D00070031816BCF333C0843F21F480916C033E
:1047E0008E7F17C0853F21F480916C038D7F11C0AF
:1047F000863F21F480916C038B7F0BC0873F21F4AF
:1048000080916C03877F05C0883F31F480916C03F1
:104810008F7E80936C0313C08D3F21F480916A03D7
:104820008E7F0BC08E3F21F480916A038D7F05C07F
:104830008F3F29F480916A038B7F80936A03809174
:104840006D0381110EC080916E0381110AC08091A9
:104850006F03811106C080917003811102C0109214
:104860006B0308958091620383FF7EC08BE295E025
:104870000E94DD0580916C031F928F9386E295E084
:104880009F938F930E94760684E295E00E94DD0557
:1048900080916D03282F082E000C330B3F938F93CC
:1048A00081E295E09F938F930E9476068FE195E0D9
:1048B0000E94DD0580916E03282F082E000C330B1B
:1048C0003F938F938CE195E09F938F930E947606A0
:1048D0008AE195E00E94DD0580916F03282F082E64
:1048E000000C330B3F938F9387E195E09F938F9359
:1048F0000E94760685E195E00E94DD0580917003B7
:10490000282F082E000C330B3F938F9382E195E004
:104910009F938F930E9476068FE095E00E94DD05BD
:1049200080916B031F928F938CE095E09F938F9300
:104930000E9476068AE095E00E94DD0580916A0378
:104940001F928F9387E095E09F938F930E94760646
:1049500084E095E00E94DD058DB79EB74C960FB6BA
:10496000F8949EBF0FBE8DBF8CE693E00E94141595
:104970000E941B22909369038093680308951F93FC
:10498000CF93DF9380916803909169030E94332253
:10499000AC0190916B03992321F020912B0130E021
:1049A00006C020912C018AE0289F90011124421713
:1049B000530708F485C080916D03C0916E03D091B8
:1049C0006F0310917003811107C0C11175C0D1111F
:1049D00073C0111171C074C09F3F19F09F5F909315
:1049E0006B03181624F40E94C32280936D038091F8
:1049F0006D0387FF05C00E94C322819580936D03DC
:104A00001C1624F40E94C32280936E0380916E03CF
:104A100087FF05C00E94C322819580936E03609139
:104A20006D03662331F1C0916E03CC2311F1062E84
:104A3000000C770B880B990B0E94742923E333E356
:104A400043E35FE30E94D8290E943C2960936D03F1
:104A50006C2FCC0F770B880B990B0E94742923E3E2
:104A600033E343E35FE30E94D8290E943C2960932B
:104A70006E031D1624F40E940C2380936F03809113
:104A80006F0387FF05C00E940C23819580936F03FD
:104A9000111624F40E940C238093700380917003FC
:104AA00087FF05C00E940C23819580937003DF91DE
:104AB000CF911F910C9432249F3F09F08FCFA0CF4C
:104AC000DF91CF911F910895ECE6F3E085E0DF01DF
:104AD0001D928A95E9F710926B0310926A0308956C
:104AE0008EE497E00E94DD051F9281E08F931F9274
:104AF00085E08F9380E097E09F938F930E947606E6
:104B00000F900F900F900F900F900F90089583309B
:104B1000E9F128F4813061F0823009F1089585309F
:104B200009F462C008F449C0863009F474C00895DD
:104B300080912C01262F30E0280F311D2F3F3105A9
:104B400024F4680F60932C0103C08FEF80932C0135
:104B500080912C011F928F9389E396E072C080911F
:104B60002B01262F30E0280F311D2F3F310524F473
:104B7000680F60932B0103C08FEF80932B0180910E
:104B80002B011F928F9387E296E05BC080912A01F0
:104B9000262F30E0280F311D2F3F310524F4680FF8
:104BA00060932A0103C08FEF80932A0180912A012C
:104BB0001F928F9384E196E044C080912901262FB3
:104BC00030E0280F311D2F3F310524F4680F60932A
:104BD000290103C08FEF80932901809129011F9241
:104BE0008F938FEF95E02DC080912801262F30E024
:104BF000280F311D2F3F310524F4680F60932801E1
:104C000003C08FEF80932801809128011F928F931A
:104C100086EE95E016C080912701262F30E0280F00
:104C2000311D2F3F310524F4680F6093270103C025
:104C30008FEF80932701809127011F928F938BEC38
:104C400095E09F938F930E9476060F900F900F90A0
:104C50000F900895833081F128F4813059F082302B
:104C6000D1F00895853009F449C0B8F1863009F4CF
:104C700056C0089580912C01681720F4861B8093FC
:104C80002C0102C010922C0180912C011F928F9355
:104C90008CEB95E054C080912B01681720F4861BA3
:104CA00080932B0102C010922B0180912B011F9247
:104CB0008F938AEA95E043C080912A01681720F417
:104CC000861B80932A0102C010922A0180912A013A
:104CD0001F928F9387E995E032C080912901681770
:104CE00020F4861B8093290102C010922901809133
:104CF00029011F928F9382E895E021C080912801BD
:104D0000681720F4861B8093280102C010922801A6
:104D1000809128011F928F9389E695E010C08091C1
:104D20002701681720F4861B8093270102C0109288
:104D30002701809127011F928F938EE495E09F9326
:104D40008F930E9476060F900F900F900F9008950A
:104D5000CF93C82F1F928F9383E598E09F938F93F3
:104D60000E94760681E090E0A0E0B0E0BC01CD01B9
:104D700004C0660F771F881F991FCA95D2F70E943B
:104D8000491F0F900F900F900F90CF910C94CD175B
:104D9000CF93873288F58E3108F00BC18E3009F43D
:104DA00087C0D8F4873009F460C08B3009F44FC055
:104DB000863009F002C180916203817F8E7F8093EB
:104DC000620388E598E00E94DD0589E09BE00E948F
:104DD000DD0581E08093720346C0863109F4B0C0DE
:104DE00020F4803109F47AC0E8C0893109F491C017
:104DF0008B3109F449C0E1C0883349F150F489325C
:104E000009F4D5C0853309F4D2C0873209F0D5C082
:104E1000CEC0833409F4CBC028F48A3308F4CDC063
:104E20008953C8C0883409F0C8C00E94CD1788EFE4
:104E30009AE00E94DD052FEF83ED90E32150804042
:104E40009040E1F700C000000E9468220CC08FE78C
:104E500098E041C08FED9AE00E94DD0580916203E9
:104E6000816080936203C1E0ADC080916203C82F6E
:104E7000C17080FFEFCF8BEE9AE00E94DD0580913C
:104E80006203817F8E7F3FC09091620391FBCC27AC
:104E9000C0F981E0C827892FC0FB81F980936203A4
:104EA000CC2319F082ED9AE029C084EC9AE013C07B
:104EB0009091620392FBCC27C0F981E0C827892F2B
:104EC000C0FB82F980936203CC2319F085EB9AE052
:104ED00015C085EA9AE00E94DD05C5CF9091620376
:104EE00093FBCC27C0F981E0C827892FC0FB83F949
:104EF00080936203CC2351F089E99AE00E94DD059A
:104F0000809162038160809362035CC08CE89AE0C8
:104F1000E2CF8DE79AE00E94DD058AE59AE00E94E3
:104F2000DD0585E19AE00E94DD058DEE99E00E94A5
:104F3000DD0588EA99E00E94DD058DE799E0CBCF99
:104F40008FE699E00E94DD050E94BF141F928F93A7
:104F500085E599E09F938F930E94760680912401C6
:104F60001F928F938EE399E09F938F930E94760612
:104F700080917F021F928F938BE299E09F938F9392
:104F80000E9476060E9427229F938F937F936F93B0
:104F900084E199E09F938F930E9476068DB79EB728
:104FA00042960FB6F8949EBF0FBE8DBF5CCF80E0D7
:104FB00001C08D510E94A82656CF82E199E00E943F
:104FC000DD05C0E08C2FCF91089580E008950C940A
:104FD000E527CF93C82F80917203813069F020F0CC
:104FE000823009F449C040C167E08FE00E942A1670
:104FF000882309F43FC106C067E08FE00E942A16AB
:10500000882361F08C2F0E94E727811104C08C2F28
:105010000E94C8262FC081E090E02CC08C2F0E94F7
:10502000E527811126C0C431E1F070F4CB3081F066
:10503000C031D1F40E9470258BE498E00E94DD0518
:1050400082E08093720315C0C93259F0C83361F40D
:1050500088E598E00E94DD058FE498E00E94DD0578
:1050600008C01092720304C189E498E00E94DD0533
:10507000FFC081E08170FEC0C43228F5CE3108F057
:10508000C1C0CB30A1F1D0F4C73009F0D3C08EE15C
:1050900080932C0182E380932B018AE080932A0184
:1050A00084E18093290188E08093280188E280933D
:1050B00027018FEE96E00E94DD05BFC0C33149F1A4
:1050C000C431C1F0B7C0CB3409F4A9C028F4C93247
:1050D00089F0C83361F0AEC0C13509F49EC0C23555
:1050E00009F499C0CE3409F0A5C06AE09EC00E94C0
:1050F0007025A3C080917103882319F01092710369
:105100009CC08CEF96E00E94DD0581E080937203E5
:10511000B1C086ED96E00E94DD0584EC96E00E9429
:10512000DD0580912C011F928F9381EC96E09F9377
:105130008F930E9476068FEB96E00E94DD058DEA44
:1051400096E00E94DD0580912B011F928F938AEAE1
:1051500096E09F938F930E94760688EA96E00E94DD
:10516000DD0589E996E00E94DD0580912A011F9204
:105170008F9386E996E09F938F930E94760684E949
:1051800096E00E94DD0583E896E00E94DD058091AF
:1051900029011F928F9380E896E09F938F930E943E
:1051A00076068EE796E00E94DD0589E696E00E948D
:1051B000DD05809128011F928F9386E696E09F93EC
:1051C0008F930E94760684E696E00E94DD058DE4CA
:1051D00096E00E94DD05809127011F928F938AE45B
:1051E00096E09F938F930E94760688E496E00E9453
:1051F000DD058DB79EB748960FB6F8949EBF0FBEDB
:105200008DBF1BC0CE51EC2FF0E0E85BFE4F8081DC
:105210008093710312C061E003C061E006C06AE0E0
:10522000809171030E94872508C0809171030E94BC
:105230002A2603C08DEE96E013C080917103882367
:1052400069F01F928F9387EE96E09F938F930E9451
:1052500076060F900F900F900F9004C084EE96E0AA
:105260000E94DD0581E006C01092720380E002C05A
:1052700080E000CFCF9108950E9443296894B11136
:105280000C94D22908950E94B72988F09F5798F06E
:10529000B92F9927B751B0F0E1F0660F771F881F3B
:1052A000991F1AF0BA95C9F714C0B13091F00E9455
:1052B000D129B1E008950C94D129672F782F882740
:1052C000B85F39F0B93FCCF3869577956795B3957C
:1052D000D9F73EF490958095709561957F4F8F4FEB
:1052E0009F4F0895E89409C097FB3EF490958095F0
:1052F000709561957F4F8F4F9F4F9923A9F0F92F9C
:1053000096E9BB279395F695879577956795B79519
:10531000F111F8CFFAF4BB0F11F460FF1BC06F5FFF
:105320007F4F8F4F9F4F16C0882311F096E911C011
:10533000772321F09EE8872F762F05C0662371F032
:1053400096E8862F70E060E02AF09A95660F771F46
:10535000881FDAF7880F9695879597F9089557FD76
:105360009058440F551F59F05F3F71F04795880FD3
:1053700097FB991F61F09F3F79F08795089512166A
:1053800013061406551FF2CF4695F1DF08C0161616
:1053900017061806991FF1CF8695710561050894C7
:1053A0000895E894BB2766277727CB0197F90895DE
:1053B0000E94EB290C945C2A0E944E2A38F00E942D
:1053C000552A20F0952311F00C94452A0C944B2A71
:1053D00011240C94D2290E94AF2970F3959FC1F338
:1053E000950F50E0551F629FF001729FBB27F00D93
:1053F000B11D639FAA27F00DB11DAA1F649F6627E8
:10540000B00DA11D661F829F2227B00DA11D621F36
:10541000739FB00DA11D621F839FA00D611D221FF0
:10542000749F3327A00D611D231F849F600D211DD4
:10543000822F762F6A2F11249F5750409AF0F1F057
:1054400088234AF0EE0FFF1FBB1F661F771F881FC0
:1054500091505040A9F79E3F510580F00C94452A89
:105460000C94D2295F3FE4F3983ED4F38695779568
:105470006795B795F795E7959F5FC1F7FE2B880F66
:10548000911D9695879597F9089597F99F6780E8FC
:1054900070E060E008959FEF80EC089500240A9486
:1054A0001616170618060906089500240A941216FF
:1054B0001306140605060895092E0394000C11F432
:1054C000882352F0BB0F40F4BF2B11F460FF04C0DF
:1054D0006F5F7F4F8F4F9F4F089597FB072E16F4F6
:1054E000009407D077FD09D00E94872A07FC05D0D9
:1054F0003EF4909581959F4F0895709561957F4FEB
:105500000895EE0FFF1F0590F491E02D0994AA1B5A
:10551000BB1B51E107C0AA1FBB1FA617B70710F09E
:10552000A61BB70B881F991F5A95A9F780959095D0
:0A553000BC01CD010895F894FFCFEF
:10553A00FFFFA514000069FFFF27E78C000000FFAA
:10554A00FF9464000576010000FF740C040DE10C61
:10555A00AB0C770C0158032808140A321E796573BC
:10556A00006E6F00404D362270042304ED03CB0316
:10557A00570370038903A2030102030405060708FF
:02558A00090016
:106800000000EA44E944E2440400050006000700F1
:10681000080009000A000B000C000D000E000F001C
:1068200010001100120013001400150016001700CC
:10683000180019001A001B001C001D001E001F007C
:10684000200021002200230024002500260027002C
:10685000280029002A002B002C002D002E002F00DC
:10686000300031A232003300340035A13600370049
:10687000380082003A003B003C003D003E003F00F3
:1068800040004100420043004400450046004700EC
:10689000480049004A004B004C004D004E004F009C
:1068A00050005100520053002E0054005500560075
:1068B000580059005A005B005C005D005E005F00FC
:1068C0006000610062006300640000005700000087
:1068D000CD440000000000000000000000000000A7
:1068E0000000000000006620000000000000000022
:1068F000E000E100E300E200E400E500E600000063
:106900000000010001000100EA4401000100E2442E
:106910000100010001000100460001004A004B0097
:10692000010001004700480001000100E9440100A6
:106930000100010001000100010001003A003B00DC
:106940003C003D003E003F0040004100420043004B
:10695000010035004C0001000100440045005200D8
:1069600049000100010050004F0029004D004E0079
:1069700051000100010001000100010001000100BF
:1069800001000100010001000100010001000100FF
:1069900001000100010001000100010001004D00A3
:1069A0004A004E004B0001000100010001000100FF
:1069B00001000100010001000100010001000100CF
:1069C00001000100010001000100000001000000C1
:1069D00001000000000000000000000000000000B6
:1069E00000000000000001000000000000000000A6
:1069F0000100010001000100010001000100000090
:106A00000000010001000100EA4401000100E2442D
:106A10000100010001000100460001004A004B0096
:106A2000010001004700480001000100E9440100A5
:106A30000100010001000100010001003A003B00DB
:106A40003C003D003E003F0040004100420043004A
:106A5000010035004C0001000100440045005200D7
:106A600049000100010050004F0029004D004E0078
:106A700051000100010001000100010001000100BE
:106A800001000100010001000100010001000100FE
:106A900001000100010001000100010001004D00A2
:106AA0004A004E004B0001000100010001000100FE
:106AB00001000100010001000100010001000100CE
:106AC00001000100010001000100000001000000C0
:106AD00001000000000000000000000000000000B5
:106AE00000000000000001000000000000000000A5
:106AF000010001000100010001000100010000008F
:00000001FF
